:0300000002036494
:03004300020100B7
:1001000002013C000201580002011800020129000E
:10011000020120000201180032E591C2E4F59122AB
:10012000C0E0C2003119D0E032C0E0E5874401F5FB
:10013000870000003119D0E032C2DC32C0D0C0E00C
:10014000C082C08312016931197401907FABF0D075
:1001500083D082D0E0D0D032C0D0C0E0C082C08393
:090160001204003119740280E25E
:10016900907FE8E0A2E79202545C7051E0A2E0823D
:10017900E1404A30E50274035403C4F540A3E05456
:100189000F45401201D52001343002182003209078
:100199007F027846754003E6F0158218D540F8E6E7
:1001A900907FB5F0754002907FB4E04540F022851C
:1001B9008240E583907FD4F0E540A380E675400353
:1001C90080E5E02582F58250020583229001FA310B
:1001D900CCE09001FA31CCC082C0837845E4F618AE
:1001E900F6187601907FEAE0F5F0A3E0C201C203B8
:1001F900226D404040404081406A74404040404048
:1002090040714040404040A540404040404040404F
:1002190040714240404040404040404040404040A2
:1002290040405663404040404040435D404040406C
:1002390040D201223000FA907FC5F0907FAAE054A5
:100249000160FBF00203EB3000E70876182230006A
:10025900E0F541223000DA08A641223000D50876BF
:100269000122760222E5F060061470C5D20022C28E
:100279000022D203149002C560B9149002D760B36A
:100289001470AE900318E5F0601EF54031CBE060C4
:10029900A0E5401480F2D203C394219002E960934F
:1002A900149002F9608D8089E0FFF5F07800F2087A
:0C02B900A3E0DFFAD0E0D0E0E5F021A9DE
:1002C500120101010000004042420001000101024B
:1002D5000001090222000101008032090400000129
:1002E50003000000092100010001221F000705810C
:1002F500034000C80600FF0901A1011901290215E3
:100305000026FF0075089507810219012902950C41
:100315009102C0040309042C035500530042002038
:1003250000440065007300690067006E002000420C
:1003350000790020004500780061006D0070006CB8
:100345000065001A03540065006D007000650072B9
:0F03550000610074007500720065007300000005
:100364007581EB75927F78D6E254F3F21203DAE2E8
:100374004406F2E4F52004F542F5497893E4F27971
:100384009CF4F30809E2540FF2E344F0F30809E2A1
:1003940054F0F2E3440FF378967404FE74014EF2C1
:1003A4007D0C1204487D0A120448FA7401F2754067
:1003B400141203DDEA7DEE120448CEC33370DCE48C
:1003C40078ACF208F2087403F2087401F275E801DB
:1003D40075A8C00080FD75406490FB50A3E582457C
:1003E4008370F9D540F322907EC078467F0CE0F606
:0C03F400A308DFFA22907FB77407F02204
:10040000D5496F754964907E8078967404FE7401B6
:100410004EF27DAA120448120457EEC33370EE90D8
:100420007E807846794C7D007E017F06E0C3965041
:1004300003ED4EFDE0C3974003ED4EFDEE23FEA31A
:100440000809DFE8EDF080B17F0814F2CD13CD92FA
:10045000E1F204F2DFF4227F09FA799C74FDF3796A
:1004600099EA14F200E3A2E1CD13CD04F2DFF3ED3B
:03047000F0A322D4
:00000001FF
